:020000002136A7
:1D000300C000C0E07422253D253DF8C2AF863B08863CD2AFD203D0E0D000C2A832C0
:020023002103B7
:20002B00C2CFC0E0C0F0C082C083C0D0752100E522700FE523700B7C00A2B79286B3928767
:20004B000199D208E52615267044E514C39CFB50027B00E5237007E514C395225001E4F5EB
:20006B00F0C39BEB4002E5F08510F0A42528F526E522700215231522BCFF027CFE0CE52A5A
:20008B00252CF52C540F252E90033B93F580E524700FE525700B7D00A2B792A6B392A7014F
:2000AB00F8D209E52715277044E515C39DFB50027B00E5257007E515C395245001E4F5F033
:2000CB00C39BEB4002E5F08511F0A42529F527E524700215251524BDFF027DFE0DE52B25B8
:2000EB002DF52D540F252F90033B93F5A0D0D0D083D082D0F0D0E03230982FC0E0C0D0C229
:20010B0098A79930000AB74207200216D202893A300207B70D04C202D20109430180EAB5EF
:20012B000104D2B380FED0D0D0E032758E0175813E758780758922E5B0C454079003339349
:20014B00F58DF58BD288D28E759852783D760018B801FAD2007A8079807402F510F51174C9
:20016B0032F512F51375CBFF75CA4775C80475A8B075B820C2B3318F31AF51FE80F8318F77
:20018B003000FB22EAB50101223099FDC2998A008699C200B60D02D2000A4302802285F0BB
:2001AB003AC2012220010122053A433A80A83AE6C3943040E9F539940950E3753108853AB2
:2001CB00F0053A433A80A83AE6C3943040D0940A50CCD531EC85F03A753808053A433A803D
:2001EB00A83AE6C39430C0E0E538242FF8D0E0F6D538E8E53375F00AA42532F532E53575CA
:20020B00F00AA4253475F064A42532F532E435F0F53375F010E536A4F53475F027E536A418
:20022B00F53585F036E5342532F532E5333535F533E537F5345406232323F535E5375401FA
:20024B0075370160037537FFE539B40021E512C395285001E48510F084C2CA853222853313
:20026B002385302885352E85372AF51441D9B40121E513C395295001E48511F084C2CA85E3
:20028B00322485332585302985352F85372BF51541D9B4040585329041D9B4050451EF41F2
:2002AB00D9B4060985343DC289D2A841D9B40717533401E5342410F8E5306016A630E534A9
:2002CB002412F8A63241D9B4080851E041D9D2CAB2B3C2012231897442712BE521712074E7
:2002EB000D712B2231897442712BE5907116740D712B2230031431897442712BE53C7116E6
:20030B00E53B7116740D712BC20322C0E0C47120D0E0712022540FB40A00400224072430ED
:20032B003099FDC299F59922FFFEFDFAF4E8D0A06064444060644440606444406064444081
:20034B0043495869636D5C4D43495869636D5C4D434249505870696263666D745C544D4668
:10036B00434249505870696263666D745C544D46E4
:00000001FF
